:020000040000FA
:0600000000000DEF00F00E
:060008009E90122A110077
:08001800FFD744D8C9D8CFD8A6
:100020001106FCE1640E116E12C018F0CECF16F06E
:10003000CF50176ED8A812C018F0C1D8CF50CE1824
:10004000E806FEE112C015F0CECF13F0CF50146ECB
:10005000D8A812C015F01650135C166E175014581D
:10006000176E18501558186E090E165ED8A0170690
:10007000D8A018061650195C17501A5818501B585B
:10008000D8A016C019F0D8A017C01AF0D8A018C070
:100090001BF019C01FF01AC01EF01BC01DF041D884
:1000A000A5D8BCD78E0EC16EE10E926EDC0E936E9B
:1000B000D00E946E0F0E956E000E966E880ED56E55
:1000C000100E806E810ECD6E196A1A6A1B6A336A31
:1000D000010E116E0DD883CF10F0020EF76E2E0EAA
:1000E000F66E45D89F809E909D80D08EF28E120035
:1000F0000A0E036E64D80306FDE18490020EF76ECB
:10010000260EF66E08008482F5CF83FF849257D8BE
:100110008482F538836E849252D80B00F552F3E155
:1001200012000A0E266E7EEC02F0D8901F361E36A4
:100130001D361F361E361D362150E8240700E824E0
:100140000700050F0700F00BE8381F26E86A1E229B
:100150001D22120019C01FF01AC01EF01D6AE1DF37
:1001600045D81200210E036E0306FEE112008490B2
:100170000800F55201E10B008482F5CF83FF8492E1
:100180008482F538836E8492EDDF84800B00F55213
:10019000F3E1120084908482EFCF83FF8492848203
:1001A000EF38836E8492DEDF8480EC50F4E112003D
:1001B0008088040603E1FA0E046E80981200F2A40F
:1001C000FED7F2CF02F0F29CF29ED6CF00F0D7CF4E
:1001D00001F0660E00269E0E012201C0D7FF00C06E
:1001E000D6FF0250C00BF212F294120000EE0EF095
:1001F0000A0E266E7EEC02F021503009ED6EE950B9
:100200000608F6E1300EEC5C03E1200EEF6E01D043
:1002100003D0E9500D08F6E100EE06F0C00E066EC0
:100220000F6AB8DF1200333228010C06000080503C
:10023000576D6178207573000000010001805655EC
:1002400001403433AB2A93240120721C9A194617BB
:100250005615B2134A1212110110100F390E7A0DF1
:10026000CD0C310CA30B220BAB0A3E0AD9097C0939
:100270002509D408890843080108C20788075107DF
:100280001D07EC06BD06910667063F061906F50533
:10029000D205B1059105730556053A051F050605FA
:1002A000ED04D504BE04A80493047E046A04570434
:1002B00045043304220411040104F103E103D303D0
:1002C000C403B603A9039C038F03820376036A0366
:1002D0005F03540349033E0334032A032003160338
:1002E0000D030403FB02F202E902E102D902D1028A
:1002F000C902C102BA02B202AB02A4029D02960276
:100300009002890283027D02770271026B0265020C
:100310005F025A0254024F024A0244023F023A026A
:10032000350231022C02270223021E021A02150294
:1003300011020D02090205020102FD01F901F50198
:10034000F101ED01EA01E601E201DF01DB01D80183
:10035000D501D101CE01CB01C801C401C101BE014B
:10036000BB01B801B501B301B001AD01AA01A701FC
:10037000A501A2019F019D019A0198019501930198
:1003800090018E018B018901870184018201800126
:100390007E017B01790177017501730171016F01A4
:1003A0006D016B01690167016501630161015F0115
:1003B0005D015B015901580156015401520151017F
:1003C0004F014D014B014A014801470145014301DD
:1003D000420140013F013D013C013A013901370131
:1003E000360134013301310130012F012D012C017F
:1003F0002A012901280126012501240122012101C8
:1004000020011F011D011C011B011A011901170107
:100410001601150114011301120110010F010E0143
:100420000D010C010B010A01090108010701060178
:1004300005010401030102010101100E266008D02C
:1004400026B6100C26B4200C26B2400C26B0800C28
:1004500026BC020C26BA040C26B8080C20C024F0D6
:10046000206A1FC023F01F6A1EC022F01E6A1DC032
:1004700021F01D6A000C216A000C010E26643BEF7E
:1004800002F0D890F76A2634F736390FF66E020E6E
:10049000F7220A001DC022F01EC021F0F5502202F2
:1004A000F4CF1DF0F3CF1EF00900F5502102F4CF78
:1004B0001FF02202F3501F26F4501E22E86A1D226C
:1004C0000A00F5502102F3501F26F4501E22E86A5C
:1004D0001D2226501E02F3CF20F0F4CF1FF01D0284
:1004E000F3501F262050215E1F50225A22AE000CCE
:1004F0001E06E86A1D5A26502126000C1DC033F046
:100500001EC034F01FC035F03DEC02F01DC033F0CA
:100510001EC034F035C01EF021C01DF03DEC02F0CD
:0E0520001EC01FF034C01EF033C01DF0000CD2
:020000040030CA
:08000000FFFAF6FEFFFFFBFF13
:00000001FF
